:10000000C828B000F839A400A40CA40C240C840760
:100010007320B0000005C3283008031C030100064C
:1000200030058006C328A01123080319A015053048
:10003000A2002730A900103029200330A900E830A1
:100040002920A90164302920A9010A3029202A0881
:100050003028A8002B08A5002A08A4008020240826
:10006000A400A2030319A011230803193A282202AD
:10007000031841282408031DA011A0194128303E6F
:10008000472808000C1E422899000314C328211990
:100090004228080083169B0083161C141A089B0A2A
:1000A000C328A901A800FF30A807031CA907031C47
:1000B000C3280330A500E5305F205328A501F63E94
:1000C000A400A509031C6A28FE300000A407031839
:1000D0006528A4070000A50F6428000024187028D4
:1000E00024187228080000308A0030080739820777
:1000F0000134023404340834103420344034803461
:10010000AB01AA011030AE00250DAA0DAB0D2808D9
:10011000AA022908031C290FAB02031896282808F5
:10012000AA0729080318290FAB070310A40DA50D72
:10013000AE0B84282408C3281030B100A501A40107
:10014000AF0CAE0C031CAA282808A4072908031822
:10015000290FA507A50CA40CAB0CAA0CB10BA02869
:100160002A08C328A400A71BB7202408C328A40971
:10017000A509A609A709A40A0319A50A0319A60A2D
:100180000319A70A08008313831203130000080051
:1001900083160F3099002030980083128030980029
:1001A000A001423083168600FD308500073083129F
:1001B0009F00BF2964305E20861564305E200614DF
:1001C00064305E20861164305E20061064305E204C
:1001D0000800DA20851464305E2036214821061B91
:1001E0002529851913294D304220413042204730BE
:1001F00042204E30422045304220543042203D3093
:100200004220203042200430A100A3013508AB0079
:100210003408AA00132020304220422042204220ED
:100220000D30422024294D303407BC003508031816
:10023000013EBD004D3042203408422035084220A6
:100240003C0842203D084220EF28051D2D290610BC
:1002500086150A30512086110800E92885100A30D9
:100260005E20080085140A305E2008000B30BB00B9
:100270002E213221343084003B08003E012003103F
:10028000051803140C200130BB020318382908009C
:100290002E21322183100518831483183A14831CED
:1002A0003A102E2132218310051883148318BA14B2
:1002B000831CBA102E213221831005188314831851
:1002C0003A15831C3A112E2132218310051883140C
:1002D0008318BA15831CBA112E21322183100518F8
:1002E000831483183A16831C3A122E21322183106C
:1002F000051883148318BA16831CBA128615143095
:100300005E2008003508AF003408AE00A9012D308A
:10031000A8009C20C1002B08C2004208BF00C001F9
:100320000310BF0C4108C30001304205C40044085B
:10033000AF004308AE00A9010A30A8009C20C3000A
:100340002B08C4004408C500C6010310C50C4308AF
:10035000C10001304405C20001304202031CBE2925
:100360004508093A4604031DBB29BF0A0319C00A00
:10037000C601C501BE29C50A0319C60A0800061030
:100380000330A900E8305220C901C801C701861313
:1003900000304A20BE0086158514B501B401143022
:1003A0005E200519D429E920861114305E203621FB
:1003B0008618FF293508AB003408AA00AC01AD014E
:1003C000013EB600F030B7002B0803182B0FB7071B
:1003D000FF30B8002C0803182C0FB807FF30B90005
:1003E0002D0803182D0FB9073908A7003808A600F3
:1003F0003708A5003608B220B4002508B500023041
:100400004902031C0F2A4808A5004708A400A901B7
:100410004908A8008020CB002508CC00132A4808F2
:10042000CC004708CB0035084C02031C262A031DCC
:100430001D2A34084B02031C262A34084B02CD0027
:100440003508031C013E4C02CE002E2A4B08340214
:10045000CD004C08031C013E3502CE00CE08031D22
:10046000352A0A304D02031C3C2A3508C8003408DE
:10047000C7000130C900472A0F3049020318472A34
:100480003408C70735080318013EC807C90A4821C0
:1004900001305120BA1D4E2A0612502A06160616A1
:1004A0003A1E542A8612562A86168616061BE42AF7
:1004B0008519B42A8221BE08031D872A41304220B3
:1004C0005A304220493042204D304220553042209F
:1004D0005430422048304220203042203D304220DB
:1004E000203042200430A100A3014008AB003F08A7
:1004F000AA0013202E304220A3014608AB00450875
:10050000AA001320203042200D304220B32A45306B
:1005100042204C304220453042205630422041306B
:10052000422054304220493042204F3042204E3049
:100530004220203042203D304220203042200430F2
:10054000A100A3014008AB003F08AA0013202E30F1
:100550004220A3014608AB004508AA001320203022
:1005600042200D304220E12A41304707B2004808BE
:100570000318013EB30049083207BC0033080318D2
:10058000013EBD00BE08031DD22A4130422047086B
:10059000422048084220490842203C0842203D08A9
:1005A0004220DE2A453042204708422048084220A7
:1005B000490842203C0842203D084220C901C801A8
:0E05C000C701061BE42AE12ACB296300E52AC5
:02400E00223F4F
:024200000000BC
:00000001FF
